:020000040000FA
:020000001228C4
:08000800FE00030E8301C40099
:100010000A08C5008A010408C7004008C200410858
:10002000C3006E284E2883125F100C1083160C102C
:1000300008001320831290101C16CF3010051038C2
:1000400090001013101510148B170B1708005F1C6D
:100050002D28FF30C000C10008000E08C0000F08A6
:10006000C10008004D088E004E088F005F100C1074
:1000700083160C14080083120C1C412813208312D1
:100080008C164208C0004308C10047088400450898
:100090008A00440E8300FE0E7E0E090083160515AD
:1000A000E0298312D5011320F0308312150504389E
:1000B0009500DF118C1283168C16080051208312D4
:1000C000DF100B178B1708008312DF1C6C285908F0
:1000D000DB00DF1040140800401008008C1E3B2895
:1000E0008C12DF1D7528DF117628DF15DF1D7D28B6
:1000F000F0301505053895008128F03015050438D5
:100100009500272083124008D3004108D400CD0178
:10011000CE01322083125508031D91280130D500ED
:100120003B285503031DB32869305402031D9A2848
:1001300078305302C811031D0318C815AF3054029C
:10014000031DA428C83053024812031D031C48167F
:10015000C816C819481EC812C81EB1280230D500DA
:100160003B2851203B2802305502031DF92834302A
:100170005402031DBD28BC305302C813031D0318CD
:10018000C81757305402031DC728E43053024910E2
:10019000031D031C4914C914C81B491CC910C91CE0
:1001A000DA285F15CF01D001D101D201D601033089
:1001B000D5003B281A305402031DE028603053025A
:1001C0004911031D031849152B305402031DEA2859
:1001D000F0305302C911031D031CC91549164919F2
:1001E000C91D4912491EF7280530D5003B2851206A
:1001F0003B2803305502031D68295F1D1D29063069
:100200005402031D0529973053024913031D031897
:1002100049170A305402031D0F29FC305302C91339
:10022000031D031CC9174A14491BC91F4A104A1C45
:100230001B295F1157295120572906305402031DED
:10024000232997305302CA10031D0318CA140A3019
:100250005402031D2D29FC3053024A11031D031CB7
:100260004A15CA15CA184A1DCA11CA1D39295F156F
:10027000572912305402031D3F293C3053024A12C1
:10028000031D03184A1620305402031D4929F43077
:100290005302CA12031D031CCA164A174A1ACA1E61
:1002A0004A134A1F56294F145F15572951208312AC
:1002B0005F1D3B28D60A20305602031D62290430F8
:1002C000D5003B280310CF0DD00DD10DD20D3B280A
:1002D00004305502031DBE2906305402031D722945
:1002E00097305302CB10031D0318CB140A3054026D
:1002F000031D7C29FC3053024B11031D031C4B15BD
:10030000CB15CB184B1DCB11CB1DBC294F08DA00E8
:100310005008CF005108D0005208D100D2014F0838
:10032000D9005008CF005108D0005208D100D201A6
:100330004F08D8005008CF005108D0005208D10013
:10034000D2014F08D700FF30DA06FF30D806570831
:1003500058024B1203194B1659085A02CB120319B3
:10036000CB164B174B1ACB1E4B134B1FBA29DF145E
:1003700051203B2851203B2851203B280530550275
:10038000031D3B2806305402031DC8299730530231
:100390004C10031D03184C140A305402031DD229BB
:1003A000FC305302CC10031D031CCC144C154C180C
:1003B000CC1C4C114C1DDE2951203B2851203B28E0
:1003C0008113373095009F0183129F019A019C0190
:1003D000831685120512051485142A2AFD167D0838
:1003E000831285007D167D088500DC01DD01080093
:1003F0007D167D088500831203132F30C000A930BD
:10040000C1000A128A11C10B012A0A128A11C00BFB
:10041000FF29FD127D0885003030DC007530DD00DD
:100420000800FD167D088500831203132F30C000DD
:10043000A930C1000A128A11C10B1A2A0A128A11A4
:10044000C00B182A7D127D0885003030DC00753025
:10045000DD000800EE2119205E208312DE015F120C
:100460005F13DF16DF17831203135F30C000033002
:10047000C1000A128A11C10B392A0A128A11C00B53
:10048000372A000000005C085D0403194C2ADC03D5
:100490005C0A0319DD034D2AEE2164208312E0106B
:1004A0004018E014E01C642A02305B02031D5A2A43
:1004B000EE21642A62305B02031D602AF821642A5F
:1004C000A8305B020319112283125E0803196A2AFD
:1004D000DE03332A05187E2A5F1A722A5F16193046
:1004E000DE00802ADF1E7B2A5C085D04031D7A2A59
:1004F000F8217B2AEE218312DF12802A5F12DF1699
:100500008518942A5F1B882A5F171930DE00332A6A
:10051000DF1F912A5C085D04031D902A1122912A95
:0E052000EE218312DF13332A5F13DF17332A15
:02400E00C43CB0
:00000001FF
